:0200000480007A
:100000006F008004732F2034930F80006308FF0378
:10001000930F90006304FF03930FB0006300FF038E
:10002000130F000063040F0067000F00732F2034CC
:1000300063540F006F00400093E19153171F0000BD
:1000400023223FFC6FF09FFF93000000130100008C
:10005000930100001302000093020000130300004C
:100060009303000013040000930400001305000034
:10007000930500001306000093060000130700001C
:100080009307000013080000930800001309000004
:1000900093090000130A0000930A0000130B0000EC
:1000A000930B0000130C0000930C0000130D0000D4
:1000B000930D0000130E0000930E0000130F0000BC
:1000C000930F0000732540F16310050097020000B4
:1000D000938202017390523073500018970200000F
:1000E0009382020273905230B70200809382F2FF33
:1000F0007390023B9302F0017390023A73504030C8
:100100009702000093824201739052307350203066
:100110007350303093010000970200009382C2EECA
:1001200073905230130510001315F501634C050050
:100130000F00F00F930110009308D0051305000085
:100140007300000093020000638A02007390521053
:10015000B7B2000093829210739022307350003037
:10016000970200009382420173901234732540F18C
:1001700073002030B70000801301000033D7200047
:10018000B70300809301200063187756B700008002
:100190001301100033D72000B70300409301300053
:1001A000631C7754B70000801301700033D7200020
:1001B000B70300019301400063107754B70000803B
:1001C0001301E00033D72000B70302009301500071
:1001D00063147752B7000080938010001301F00180
:1001E00033D720009303100093016000631677500B
:1001F0009300F0FF1301000033D720009303F0FFBA
:1002000093017000631A774E9300F0FF1301100002
:1002100033D72000B70300809383F3FF930180005E
:10022000631C774C9300F0FF1301700033D720005C
:10023000B70300029383F3FF93019000631E774A94
:100240009300F0FF1301E00033D72000B703040050
:100250009383F3FF9301A0006310774A9300F0FFAC
:100260001301F00133D72000930310009301B00075
:1002700063147748B72021219380101213010000E6
:1002800033D72000B7232121938313129301C00099
:1002900063147746B72021219380101213011000B8
:1002A00033D72000B7939010938303099301D000B4
:1002B00063147744B720212193801012130170003A
:1002C00033D72000B7434200938323249301E000F7
:1002D00063147742B7202121938010121301E000AC
:1002E00033D72000B7830000938343489301F00085
:1002F00063147740B7202121938010121301F0017D
:1003000033D7200093030000930100016316773E6A
:10031000B720212193801012130100FC33D7200055
:10032000B723212193831312930110016316773CA5
:10033000B720212193801012130110FC33D7200025
:10034000B793901093830309930120016316773AC2
:10035000B720212193801012130170FC33D72000A5
:10036000B743420093832324930130016316773807
:10037000B7202121938010121301E0FC33D7200015
:10038000B783000093834348930140016316773697
:10039000B7202121938010121301F0FF33D72000E2
:1003A000930300009301500163187734B700008075
:1003B00013017000B3D02000B70300019301600166
:1003C000639C7032B70000801301E00033D120003D
:1003D000B703020093017001631071329300700043
:1003E000B3D0100093030000930180016396703036
:1003F00013020000B70000801301700033D7200003
:10040000130307001302120093022000E31452FEAC
:10041000B7030001930190016310732E13020000D3
:10042000B70000801301E00033D720001300000064
:10043000130307001302120093022000E31252FE7E
:10044000B70302009301A0016318732A130200008E
:10045000B70000801301F00133D720001300000023
:100460001300000013030700130212009302200080
:10047000E31052FE930310009301B001631E732634
:1004800013020000B70000801301700033D7200072
:100490001302120093022000E31652FEB70300017C
:1004A0009301C001631A772413020000B700008093
:1004B0001301E0001300000033D7200013021200E4
:1004C00093022000E31452FEB70302009301D0010F
:1004D0006314772213020000B70000801301F001BB
:1004E000130000001300000033D720001302120095
:1004F00093022000E31252FE930310009301E001E7
:10050000631C771E13020000B70000801300000078
:100510001301700033D72000130212009302200051
:10052000E31452FEB70300019301F0016316771C38
:1005300013020000B7000080130000001301E00068
:100540001300000033D72000130212009302200092
:10055000E31252FEB703020093010002631E7718F4
:1005600013020000B7000080130000001300000019
:100570001301F00133D72000130212009302200070
:10058000E31252FE930310009301100263167716D4
:100590001302000013017000B700008033D7200061
:1005A0001302120093022000E31652FEB70300016B
:1005B0009301200263127714130200001301E0007C
:1005C000B70000801300000033D720001302120090
:1005D00093022000E31452FEB7030200930130029D
:1005E000631C7710130200001301F001B7000080B4
:1005F000130000001300000033D720001302120084
:1006000093022000E31252FE930310009301400274
:100610006314770E13020000130170001300000032
:10062000B700008033D7200013021200930220008D
:10063000E31452FEB703000193015002631E770AD0
:10064000130200001301E00013000000B700008057
:100650001300000033D72000130212009302200081
:10066000E31252FEB703020093016002631677089B
:10067000130200001301F00113000000130000003A
:10068000B700008033D7200013021200930220002D
:10069000E31252FE9303100093017002631E77046D
:1006A0009300F00033511000930300009301800287
:1006B000631471049300000233D10000930300021D
:1006C00093019002631A7102B3500000930300007B
:1006D0009301A00263927002930000403711000062
:1006E0001301018033D02000930300009301B00276
:1006F00063147000631030020F00F00F638001007C
:100700009391110093E111009308D0051385010026
:10071000730000000F00F00F930110009308D00544
:100720001305000073000000731000C000000000FB
:0C073000000000000000000000000000BD
:1010000000000000000000000000000000000000E0
:1010100000000000000000000000000000000000D0
:1010200000000000000000000000000000000000C0
:1010300000000000000000000000000000000000B0
:081040000000000000000000A8
:040000058000000077
:00000001FF
